:1000000000308A006D290000831A0A288E00030E32
:100010008F000F2883128E00030E8F008F148E0E18
:10002000040890000C0891000D08920083128B1EAA
:100030001B280B1989281008840011088C0012084D
:100040008D000F0E830083120E0E8F188316090089
:100050000A108A100A1182070A3443347234653454
:1000600061347434693476346534203443346F3405
:100070006E34743472346F346C34203443346F34DF
:100080006E346334653470347434733420344D34D6
:1000900069346E3469342D34443449344F340A346D
:1000A000763431342E34303420344A3475346C3460
:1000B0007934203431343934393438340A34003422
:1000C0000A108A100A1182070A34413464346434F5
:1000D0007234653473347334203473346534743457
:1000E000203474346F342034443449344F3425344C
:1000F00063340A3400340A108A100A11820720344B
:10010000443449344F342534633420344434503437
:100110000034051E8E28FF308100EC2827308C002B
:100120008C0B902800000000BE013E08073C031C19
:10013000B728BF01051ABF0A000000000000051E15
:10014000A228BF0A000000000000051EA828BF0A60
:10015000000000000000BF18AF280310B0280314EF
:10016000BD0C19308C008C0BB328BE0A9528FF30CB
:100170008100AB1CCB283D08213C0319C3283D0856
:10018000233C031DCA28A7011330270784003D081C
:100190008000AB10EC28A70A2708143C031DD328C5
:1001A000AB14AB11EC282B18DC2828082702031D00
:1001B000DC28AB14AB11EC283D080D3C0319E428F6
:1001C0003D080A3C031DE7282B15AB14EC2813301F
:1001D000270784003D0880000B118A111B288B1211
:1001E0000515000085111F308C008C0BF5280000D0
:1001F000BA013A08073C031C0A290310B90C03187A
:1002000003298511042985151E308C008C0B0629C5
:10021000BA0AF9280000000000000000851500005F
:100220000B118B16FF3081001F308C008C0B1629B0
:100230000000051100343B1B22293B080F398D00BB
:10024000272927293B080F39093E8D00272900342B
:100250003808093C031C3129380830388D0036290C
:1002600036290930380240388D00362900343730BD
:100270008400000803194B2901308D008C018C0B80
:100280003F298D0B3E294A308C008C0B45290000FC
:100290000000800B3C29352BB81B5E290F308C00E9
:1002A000370E8C050A300C020318592930308C07A0
:1002B0005B2938088C070C08B900EF200F30B70510
:1002C0000A3037020318662930306829B813380815
:1002D000B7073708B900EF203F2B43308C000D30B3
:1002E00084008001840A8C0B7129A00184011F30D5
:1002F000830583168113FF306600F2306500831298
:10030000051100000514000085153830831681049E
:10031000FF308312AF008518C329B70137082820A2
:10032000B70AB900EF2033303702031D8E290608C3
:100330000739303EAA0089012A0888000B088C0082
:100340000B088D008B138316081555308900AA30D1
:10035000890088148818AA29081183128C1B0D089B
:100360008B00B70137086020B70AB900EF201330BF
:100370003702031DB2292A08B900EF200A30B9005C
:10038000EF20C129EE294430B1004930B2004F308E
:10039000B30089018316081483120808B4003408D6
:1003A000373C031CD72934082F3C031CEE2930307E
:1003B000B400890188000B088C000B088D008B139A
:1003C0008316081555308900AA30890088148818CA
:1003D000E729081183128C1B0D088B009F30AE009B
:1003E0003408AE07AB142B142B11A7010B138B137E
:1003F0008B1BF7298B160B11FF3081008B172B14E9
:10040000AB11A801AB1D062A2B194A2AAB19492AA0
:10041000AB1C0C2A2B1D492A2708063C0318492A25
:10042000AB151308233C031D192A0430AA0030140D
:100430001C2A0230AA003010A9012908033C031C21
:10044000332A3130290784000008B7002A08AA0A95
:10045000133E8400000837020319312AAB142B1114
:10046000FF29A90A1D2A301C472A1408BB001B219A
:100470000D0EB800F030B8051508BB001B21380878
:100480000D04AA000930A8002E08AA07492A07303F
:10049000A800022A2B102708AC002B11301C612A5F
:1004A0000930A9002C08290203185D2A2908A90A85
:1004B000133E84000008AA07522AAA080319612AD9
:1004C000FF291330280784000008AA00A80A133067
:1004D000280784000008203C031D6F2AA80A2A0868
:1004E0008C0053302A0203197A2A51300C02031966
:1004F000DC2A742B0230A807133028078400000878
:100500003D3C031D9F2AA80A1330280784000008D9
:10051000B700BB001B210D0EB900F030B905A80AC9
:100520001330280784000008BA00BB001B210D0807
:100530003907AF002F0866002F088600D32A013044
:10054000A900A80A1330280784000008373C031CC0
:10055000B02A13302807840000082F3C031CB12A5E
:10056000752B13302807840000080F39AA00AA0849
:100570000319BE2A0310A90DAA03B72A0230A8073F
:100580001330280784000008303C031DCF2A2908B7
:10059000FF3AAF052F0886002F086600D32A2908E6
:1005A000AF042F0866002B140000051053308C0098
:1005B0008C0BD82A0514752B0608AD0003302807CC
:1005C0002C020319152B031C152BB0100330A807A0
:1005D0001330280784000008373C031CF62A133028
:1005E0002807840000082F3C031CF72A752B1330C2
:1005F000280784000008A90029082F3C0318072BAE
:100600000310AD0CAA010318AA0AA903FC2A0130A1
:10061000AA0530302A07B5001330280784000008E7
:10062000A9002E302907B600262BB0142D0EB700D6
:100630000F30B7053708B80028210D08B5002D0880
:100640000F39B700B80028210D08B6002B14301C54
:10065000322B7130AA00350834073607AA07FF305D
:10066000AA06AA0A3230B70037292430B900EF2091
:10067000301C3F2B2A08B7003730B8004C29B7018F
:1006800037087B20B70AB900EF2004303702031D7A
:10069000402B3408B900EF202030B900EF2044305F
:1006A000B900EF205030B900EF20B018672B2E3082
:1006B000B900EF202908B900EF203D30B900EF2044
:1006C0003508B900EF200A30B900EF20732B3D3018
:1006D000B900EF203508B900EF203608B900EF2047
:0E06E0000A30B900EF20752B752BFF2963003F
:02400E00F93F78
:00000001FF
